:020000040000FA
:0400000077EF00F0A6
:08000800056ED8CF06F0E0CF31
:1000100007F00001E9CF0DF0EACF08F0E1CF09F0D9
:10002000E2CF0AF0D9CF0BF0DACF0CF0F3CF14F017
:10003000F4CF15F0FACF16F000C00FF001C010F0A9
:1000400002C011F003C012F004C013F0F2AA2CEFAA
:1000500000F0F2B455EF00F0F2A632EF00F0F2B08B
:100060005AEF00F00FC000F010C001F011C002F014
:1000700012C003F013C004F00DC0E9FF08C0EAFF8E
:10008000088E09C0E1FF0AC0E2FF0BC0D9FF0CC017
:10009000DAFF14C0F3FF15C0F4FF16C0FAFF0550D5
:1000A00007C0E0FF06C0D8FF100092948994F29434
:1000B00032EF00F09294898493948A74FF0E936EC9
:1000C000F29032EF00F0EA6A180EE96EEF500DE0A0
:1000D000020E016E006A002EFED7012EFBD7970E8E
:1000E000006E002EFED7EF2EF3D7BCEF00F0F86ABB
:1000F000D09E088EEA6AE96A700ED36ED350B89625
:100100000C0EAF6EA20EAC6E900EAB6EC150C00B5B
:100110000F09C16E070EB46EC150C00B0F09C16E3E
:10012000C290B098C69A949E93809392010EC66E28
:10013000000EC76ED190810ED56ECD6A000ECA6ECC
:10014000000ECB6EB70EB16E070EB46E9250926E6B
:10015000060E006E002EFED70000B450A19CB56ABA
:10016000FF0E936EF19EF28AF286C00EF212929208
:0C0170008972640E186EA7D7FAD703003E
:020000040030CA
:0E0000003FC8190E008781000FC00FE00F40AF
:00000001FF
